:0200000480007A
:100000001718000013080800377072421300F0E65A
:10001000B7303356938090243721562D1301210594
:10002000B77169529381313637826B731302029232
:10003000B7627473938222573753206E1303F3E62B
:10004000B773694D938313C63764646F1304341711
:10005000B744796B93843406377565741305352777
:10006000B7756E28938535F737266B6513068604BA
:10007000B76652209386461637376D6F1307C792BF
:10008000B7377069938737E62320080023221800CA
:10009000232428002326380023284800232A580038
:1000A000232C6800232E7800232088022322980224
:1000B0002324A8022326B8022328C802232AD80210
:1000C000232CE802232EF80217120000130282F7F5
:1000D00037686F6313081846B778656A938808B461
:1000E0003779282013091986B7696A619389B95647
:1000F000376A7661130A0A52B75A202E938A5AC673
:10010000377B6F63130B9BD2B77B6973938BEB02C7
:10011000378C2066130CFC96B72C6567938C9C0675
:10012000377D7365130D1D36B72D7375938DDD0601
:10013000371E293A130EAED0B77E6968938E0E3201
:10014000372F6461130F4F07B77F2075938F5F269A
:10015000232002012322120123242201232632011B
:1001600023284201232A5201232C6201232E7201EB
:1001700023208203232292032324A2032326B203F3
:100180002328C203232AD203232CE203232EF203C3
:1001900017120000130202EF232002002322120094
:1001A000232422002326320017150000130585E5BD
:1001B00097150000938505EE370610F01306C6F27A
:1001C0006306B5028326C5002320D600832685005A
:1001D0002320D600832645002320D6008326050051
:1001E0002320D600130505016FF09FFD370510F0A1
:1001F000130505F2232005000000000000000000A8
:0402000000000000FA
:10100000FFFFFFFFFFFFFFFFFFFFFFFFFFFFFFFFF0
:10101000FFFFFFFFFFFFFFFFFFFFFFFFFFFFFFFFE0
:10102000FFFFFFFFFFFFFFFFFFFFFFFFFFFFFFFFD0
:10103000FFFFFFFFFFFFFFFFFFFFFFFFFFFFFFFFC0
:10104000FFFFFFFFFFFFFFFFFFFFFFFFFFFFFFFFB0
:10105000FFFFFFFFFFFFFFFFFFFFFFFFFFFFFFFFA0
:10106000FFFFFFFFFFFFFFFFFFFFFFFFFFFFFFFF90
:10107000FFFFFFFFFFFFFFFFFFFFFFFFFFFFFFFF80
:10108000FFFFFFFFFFFFFFFFFFFFFFFFFFFFFFFF70
:040000058000000077
:00000001FF
